:03000000020D0EE0
:0C0D0E00787FE4F6D8FD75814D020D558C
:03000300020EA446
:100EA400C0E030B20CE54C700BB290B291B29280BB
:070EB40003754C32D0E0325F
:03001300020006E2
:0100060032C7
:03005300020007A1
:0100070032C6
:03005B0002000898
:0100080032C5
:030083000200096F
:0100090032C4
:100B3D00EFD394047480948040037F0122EF7061A1
:100B4D00C289900002120C7E64017004D2A880024A
:100B5D00C2A8900001120C7EFED394037480948081
:100B6D0040037F0222EEFD7C00700553B7FEC2B834
:100B7D00ED64014C700553B7FED2B8ED64024C70B4
:100B8D000543B701C2B8ED64034C700543B701D2FC
:100B9D00B8120C6564017004D2888002C2887F008F
:100BAD0022EF64017061C28B900002120C7E640111
:100BBD007004D2AA8002C2AA900001120C7EFED34C
:100BCD0094037480948040037F0222EEFD7C0070BC
:100BDD000553B7FBC2BAED64014C700553B7FBD298
:100BED00BAED64024C700543B704C2BAED64034C10
:100BFD00700543B704D2BA120C6564017004D28A31
:100C0D008002C28A7F0022EF6402701590000212EA
:100C1D000C7E64017005438F108003538FEF7F00AE
:100C2D0022EF64037015900002120C7E64017005B2
:100C3D00438F208003538FDF7F0022EF64047015F4
:100C4D00900002120C7E64017005438F40800353A7
:080C5D008FBF7F00227F0222FD
:10008600750A01E4F508F509FB7A007908FF020B09
:010096003D2C
:1008C600EFD394077480948040037F0122120C6555
:1008D600FED394037480948040037F0222EF704419
:1008E600EE700B900001120C7EF452935294120C8F
:1008F600656401700B900001120C7E4293F45294D1
:10090600120C65FE6402700A900001120C7E42937E
:100916004294EE6403700D900001120C7EFEF452B8
:1009260093EE4294EF64017046120C65FE700B90D4
:100936000001120C7EF452915292EE6401700B90FB
:100946000001120C7E4291F45292120C6564027000
:100956000A900001120C7E42914292120C656403C9
:10096600700D900001120C7EFEF45291EE4292EF51
:1009760064027046120C65FE700B900001120C7E2C
:10098600F452955296EE6401700B900001120C7EA3
:100996004295F45296120C656402700A9000011298
:1009A6000C7E42954296120C656403700D90000110
:1009B600120C7EFEF45295EE4296EF6403704612D8
:1009C6000C65FE700B900001120C7EF452B152B20F
:1009D600EE6401700B900001120C7E42B1F452B22B
:1009E600120C656402700A900001120C7E42B1423C
:1009F600B2120C656403700D900001120C7EFEF4B9
:100A060052B1EE42B2EF64047046120C65FE700BF2
:100A1600900001120C7EF452B352B4EE6401700BD6
:100A2600900001120C7E42B3F452B4120C656402BB
:100A3600700A900001120C7E42B342B4120C656437
:100A460003700D900001120C7EFEF452B3EE42B418
:100A5600EF64057046120C65FE700B900001120CD7
:100A66007EF452C952CAEE6401700B900001120C5A
:100A76007E42C9F452CA120C656402700A900001E3
:100A8600120C7E42C942CA120C656403700D9000B6
:100A960001120C7EFEF452C9EE42CAEF640670469D
:100AA600120C65FE700B900001120C7EF452CB52B4
:100AB600CCEE6401700B900001120C7E42CBF45216
:100AC600CC120C656402700A900001120C7E42CBB7
:100AD60042CC120C656403700D900001120C7EFE70
:100AE600F452CBEE42CCEF64077049120C65FF7EE0
:100AF60000700B900001120C7EF452E152E2EF649A
:100B0600014E700B900001120C7E42E1F452E2128B
:100B16000C656402700A900001120C7E42E142E20A
:100B2600120C656403700D900001120C7EFFF452E6
:070B3600E1EF42E27F002223
:100E6400750904E4F508FB7A0079087F031208C6C3
:100E74007509077508037F011208C6C290C291C2A2
:010E840092DB
:010E8500224A
:10006600120E64120086120E8612001ED2AF7B009C
:0B0076007A00793C7F02120D9A80F3A3
:060EBB00014C00014D0096
:03000B00020E1FC3
:100E1F00C0E0C0D0E54C6002154C20922DE54D602E
:100E2F00160545E54570020544C394DCE544940579
:100E3F00401E754D008019E545154570021544E5B6
:100E4F00454544700B754D0180067544057545DCAD
:050E5F00D0D0D0E0320C
:03001B0002000AD6
:01000A0032C3
:0300630002000E8A
:01000E0032BF
:03009B0002000F51
:01000F0032BE
:0300A30002001048
:0100100032BD
:10059500AD07EDD394047480948040037F0122ED70
:1005A500600302066AC28C900002120C7E64017020
:1005B50004D2A98002C2A9900001120C7EFED39438
:1005C500037480948040037F0222EEFF7E00700555
:1005D50053B7FDC2B9EF64014E700553B7FDD2B9EB
:1005E500EF64024E700543B702C2B9EF64034E7063
:1005F5000543B702D2B9120C65FEC3940374809407
:100605008040037F0222E58954FC4EF58990000362
:10061500120C7EFF7E0064017003538E7FEF4E70D7
:1006250003438E80EF64024E7005438904800353B3
:1006350089FB900004120C7E64017005438F0180D4
:1006450003538FFE900005120CD6E5F0F58C900053
:1006550005120CD6F58A900007120C7E6401700213
:10066500D28C7F0022ED64016003020737C28E90B1
:100675000002120C7E64017004D2AB8002C2AB9002
:100685000001120C7EFED394037480948040037F96
:100695000222EEFF7E00700553B7F7C2BBEF64017F
:1006A5004E700553B7F7D2BBEF64024E700543B7E2
:1006B50008C2BBEF64034E700543B708D2BB120CEA
:1006C50065FEC394037480948040037F0222EEC4C8
:1006D50054F0FFE58954CF4FF589900003120C7E45
:1006E500FF7E0064017003538EBFEF4E7003438E8F
:1006F50040EF64024E700543894080035389BF90E3
:100705000004120C7E64017005438F028003538F31
:10071500FD900005120CD6E5F0F58D900005120C44
:10072500D6F58B900007120C7E64017002D28E7F85
:100735000022ED6402707C538EEF900002120C7E55
:100745006401700543AF04800353AFFB90000312AF
:100755000C7EFED394027480948040037F0222EEC7
:10076500FF7E0064017003538EFBEF4E7003438ED2
:1007750004EF64024E7005438E088003538EF79094
:100785000004120C7E64017005438F048003538FAF
:10079500FB900005120CD6E5F0F5D6900005120C7D
:1007A500D6F5D7900007120C7E64017003438E10B6
:1007B5007F0022ED6403707C53D1F7900002120C88
:1007C5007E6401700543AF20800353AFDF900003C3
:1007D500120C7EFED394027480948040037F022223
:1007E500EEFF7E006401700353D1FDEF4E700343AD
:1007F500D102EF64024E700543D104800353D1FB4F
:10080500900004120C7E6401700543D101800353EE
:10081500D1FE900005120CD6E5F0F5D49000051236
:100825000CD6F5D5900007120C7E6401700343D1F8
:10083500087F0022ED640460030208C353D17F9052
:100845000002120C7E6401700543AF40800353AF74
:10085500BF900003120C7EFD7C00D394027480943B
:100865008040037F0222ED64014C700353D1DF9079
:100875000003120C7E700343D120900003120C7EFE
:100885006402700543D140800353D1BF9000041228
:100895000C7E6401700543D110800353D1EF9000A5
:1008A50005120CD6FDACF0ECF5D2AF058FD3900058
:1008B50007120C7E6401700343D1807F00227F0202
:0108C5002210
:100E8600E4F508F509750A01F50BF50C750DD47531
:0E0E96000ECD750F01FB7A007908FF0205955D
:1000A600EF640160030203A643BA80900029120C94
:1000B6007EFD7C00D3940374809480502DED7006F1
:1000C60053B6FB53B5FBED64014C700653B6FB43C8
:1000D600B504ED64024C700643B60453B5FBED64FB
:1000E600034C700643B60443B50490002A120C7EF6
:1000F600FD7C00D3940374809480502DED700653DC
:10010600B6F753B5F7ED64014C700653B6F743B531
:1001160008ED64024C700643B60853B5F7ED640368
:100126004C700643B60843B50890002B120C7EFDB2
:100136007C00D3940374809480502DED700653EEAA
:10014600EF53DFEFED64014C700653EEEF43DF1023
:10015600ED64024C700643EE1053DFEFED64034C82
:10016600700643EE1043DF1090002C120C7EFD7CCF
:1001760000D3940374809480502DED700653EEDF07
:1001860053DFDFED64014C700653EEDF43DF20EDF5
:1001960064024C700643EE2053DFDFED64034C70BF
:1001A6000643EE2043DF2090FECCE4F0A3F0120CD1
:1001B60065FE90FEC8E0548F4EF0900001120C7E52
:1001C600FE90FEC9E0548F4EF0900002120C7EFEA7
:1001D60090FECAE0548F4EF0900003120C7EFE9003
:1001E600FECBE0548F4EF0900027120C7E640190F7
:1001F600FEC87006E04408F08004E054F7F0900072
:1002060028120C7E640190FEC87006E04404F0805B
:1002160004E054FBF090001B120C7E640190FECCAF
:100226007006E04401F08004E054FEF090001C12D9
:100236000C7E640190FECC7006E04404F08004E07D
:1002460054FBF090001D120C7E640190FECC7006EB
:10025600E04410F08004E054EFF090001E120C7E93
:10026600640190FECC7006E04440F08004E054BF88
:10027600F090001F120C7E640190FECD7006E044E3
:1002860001F08004E054FEF0900020120C7E640120
:1002960090FECD7006E04404F08004E054FBF0903C
:1002A6000021120C7E640190FECD7006E04410F031
:1002B6008004E054EFF0900022120C7E640190FE60
:1002C600CD7006E04440F08004E054BFF090000892
:1002D600120CD6FD90FED2E5F0F0A3EDF090000AE8
:1002E600120CD6FD90FED5E5F0F0A3EDF090000CD3
:1002F600120CD6FD90FED7E5F0F0A3EDF090000EBF
:10030600120CD6FD90FED9E5F0F0A3EDF0900010AA
:10031600120CD6FD90FEDBE5F0F0A3EDF090002F79
:10032600120C7E90FEC17007E054FEFEF08005E0E0
:100336004401FEF090FEC1EEF0900030120C7E906B
:10034600FEB2F090002E120C7E90FEB1F090001AD4
:10035600120C7E90FEDEF0900032120C7E6401904C
:10036600FEDD7006E04410F08004E054EFF09000EB
:1003760033120C7E640190FEDD7006E04480F0804E
:1003860004E0547FF0900031120C7E640190FEC0B0
:100396007007E04401F002058CE054FEF002058C83
:1003A600EF6402600302059243BA8090002D120C9E
:1003B6007EFF7E00D3940374809480502DEF7006E8
:1003C60053EEBF53DFBFEF64014E700653EEBF43DB
:1003D600DF40EF64024E700643EE4053DFBFEF642A
:1003E600034E700643EE4043DF4090FEECE4F0A37C
:1003F600F0900004120C7EFF90FEE8E0548F4FF060
:10040600900005120C7EFF90FEE9E0548F4FF090AD
:100416000006120C7EFF90FEEAE0548F4FF090002B
:1004260007120C7EFF90FEEBE0548F4FF0900027F2
:10043600120C7E640190FEE87006E04408F0800429
:10044600E054F7F0900028120C7E640190FEE870EC
:1004560006E04404F08004E054FBF0900023120C04
:100466007E640190FEEC7006E04401F08004E054E6
:10047600FEF0900024120C7E640190FEEC7006E003
:100486004410F08004E054EFF0900025120C7E64D6
:100496000190FEED7006E04401F08004E054FEF0A9
:1004A600900026120C7E640190FEED7006E044106A
:1004B600F08004E054EFF0900008120CD6FF90FE96
:1004C600F2E5F0F0A3EFF0900012120CD6FF90FECA
:1004D600F5E5F0F0A3EFF0900014120CD6FF90FEB5
:1004E600F7E5F0F0A3EFF0900016120CD6FF90FEA1
:1004F600F9E5F0F0A3EFF0900018120CD6FF90FE8D
:10050600FBE5F0F0A3EFF090002F120C7E90FEC1F9
:100516007007E054FEFFF08005E04401FFF090FE16
:10052600C1EFF0900030120C7E90FEB6F090002ED7
:10053600120C7E90FEB5F090001A120C7E90FEFE14
:10054600F0900032120C7E640190FEFD7006E044CD
:1005560010F08004E054EFF0900033120C7E64013A
:1005660090FEFD7006E04480F08004E0547FF09039
:100576000031120C7E640190FEE07006E04401F04A
:0F0586008004E054FEF053BA7F7F00227F0222F0
:100D9A0043BA80EF64017039120CABFF90FED5E5BF
:100DAA00F0F0A3EFF0900002120CD6FF90FED7E508
:100DBA00F0F0A3EFF0900004120CD6FF90FED9E5F4
:100DCA00F0F0A3EFF0900006120CD6FF90FEDB8045
:100DDA003A900008120CD6FF90FEF5E5F0F0A3EF6A
:100DEA00F090000A120CD6FF90FEF7E5F0F0A3EFA0
:100DFA00F090000C120CD6FF90FEF9E5F0F0A3EF8C
:100E0A00F090000E120CD6FF90FEFBE5F0F0A3EF77
:050E1A00F053BA7F2235
:10001E00750C60E4F5357510057511DC85441A858F
:10002E00451BF522753601753801752B01753B019F
:10003E00753901FB7A0079087F021200A675440516
:03004E007545DC19
:01005100228C
:100D1A00020066E493A3F8E493A34003F68001F289
:100D2A0008DFF48029E493A3F85407240CC8C333DA
:100D3A00C4540F4420C8834004F456800146F6DFA9
:100D4A00E4800B0102040810204080900EBBE47E70
:100D5A00019360BCA3FF543F30E509541FFEE4939E
:100D6A00A360010ECF54C025E060A840B8E493A365
:100D7A00FAE493A3F8E493A3C8C582C8CAC583CA90
:100D8A00F0A3C8C582C8CAC583CADFE9DEE780BE48
:010EC1000030
:100C6500BB010689828A83E0225002E722BBFE028D
:090C7500E32289828A83E49322C0
:100C7E00BB010CE58229F582E5833AF583E022502B
:100C8E0006E92582F8E622BBFE06E92582F8E22275
:0D0C9E00E58229F582E5833AF583E493228F
:100CAB00BB010A89828A83E0F5F0A3E02250068714
:100CBB00F009E71922BBFE07E3F5F009E3192289D6
:0B0CCB00828A83E493F5F07401932209
:100CD600BB0110E58229F582E5833AF583E0F5F05C
:100CE600A3E0225009E92582F886F008E622BBFE39
:100CF6000AE92582F8E2F5F008E222E5832AF5837F
:080D0600E993F5F0A3E9932243
:00000001FF
